:10000000000003308A00052BA600841780048413A7
:10001000FA30B300B4013422A70AB00AAB01AC0134
:1000200000082605B300000000082605B4003306CA
:10003000340526060319AB0A0319AC0A3408B300C9
:10004000AF030319B0030319A70B13282B084A2A7F
:100050008030A100FE306221013062217530A8009D
:1000600030308F29A101A117B700B708031DB703CE
:10007000FE306221A30803193F28230B412880305A
:1000800052282308023A031D4728C030522823086B
:10009000033A031D4D28943052282308043A031DC7
:1000A0005328D430A300370823076229A101A117E0
:1000B000B700FE30622137086229A0112508031914
:1000C000A0150530A4002730AC0010307320033099
:1000D000AC00E8307320AC0164307320AC010A300E
:1000E00073202F087A28AB003008A8002F08A7003B
:1000F00018222708A700A4030319A0112508031933
:100100008428240203188B282708031DA011A01996
:100110008B28303E62290800CA00BB1F91282D3071
:100120006221BD0F9828BC0F9828BB0A0319BB0A8F
:10013000C201C301C401C501BB176A30BA0703106D
:10014000BB0CBC0CBD0CC50CC40CC30CC20CBA0F50
:100150009F283D083A02BD07BA023C083B02BC0793
:10016000BB02A501EB202E306221CB010310420D12
:10017000BD00430DBC00440DBB00450DBA00CB0DC6
:100180000310BD0DBC0DBB0DBA0DCB0D4208BD0754
:1001900043080318430FBC0744080318440FBB0768
:1001A00045080318450FBA070318CB0F0310BD0D00
:1001B000BC0DBB0DBA0DCB0D4B08303E62213D0886
:1001C000C2003C08C3003B08C4003A08C500CA0B83
:1001D000B52803104A2AA0112508031DF228A015EE
:1001E0000A30A5003D08AA003C08A9003B08A80069
:1001F0003A08A700A401B201B101B0010A30AF0072
:100200009E21A40A24082502031DFB282F08031D94
:10021000A011A01D0D29250B10292F08303E6221A9
:10022000A50BF2284A2AB40006118611831606117E
:1002300086110F30860583123408A0183D293E3000
:10024000A80080308F213330B30051211330A80033
:1002500088308F21512164308E21512164308E21CC
:100260002230B300512128303C210C303C21063093
:100270003C21A01434083D292014B300201C4B2934
:100280008611033C031C502950210730A800D030B0
:100290008F21031408002014FE3C031960298615E1
:1002A000201C201006150F3086053308F03986040F
:1002B00000000611B30E00002018512932308E21A3
:1002C00034084A2AA11B13290800A400A20124080B
:1002D00003178D000313250803178F0078210319D6
:1002E0004A2A6221A40A0319A50AA20F67294A2AE9
:1002F000831603178C170C140000000083120C08DF
:100300004A2AAC01AB00FF30AB07031CAC07031C4F
:100310004A2A0330A800E6308F218329A801FC3E39
:10032000A700A809031C9A29FF300000A70703189B
:100330009529A7070000A80F942908002A0832066B
:100340008039B400AA1FAF29A709A809A909AA09D9
:10035000A70A0319A80A0319A90A0319AA0AB21FAE
:10036000BC29AF09B009B109B209AF0A0319B00A33
:100370000319B10A0319B20AAB01AC01AD01AE0118
:10038000BE01BF01C001C1013208310430042F0495
:100390000319FA292030B3000310A70DA80DA90DE9
:1003A000AA0DBE0DBF0DC00DC10D32084102031DC7
:1003B000E32931084002031DE32930083F02031DF1
:1003C000E3292F083E02031CF4292F08BE0230083F
:1003D000031C300FBF023108031C310FC00232086A
:1003E000031C320FC1020314AB0DAC0DAD0DAE0DED
:1003F000B30BCC29B41F072AAB09AC09AD09AE0970
:10040000AB0A0319AC0A0319AD0A0319AE0A3E0878
:10041000AF003F08B0004008B1004108B2002B080F
:10042000A7002C08A8002D08A9002E08AA004A2A17
:10043000B001AF011030B300280DAF0DB00D2B0887
:10044000AF022C08031C2C0FB00203182E2A2B0815
:10045000AF072C0803182C0FB0070310A70DA80D29
:10046000B30B1C2A270808001030B900A801A70107
:10047000B40CB30C031C422A2B08A7072C08031842
:100480002C0FA807A80CA70CB00CAF0CB90B382A7E
:100490002F08080083138312031308004308C000C9
:1004A0004706CE004208003A031D4608003A0319E9
:1004B000A02AC2077E30031C612AC2020318A22AA6
:1004C000642AC202031C9F2A4508BE004408BF00DC
:1004D000C017C717C501C401C3011830CD00C00C37
:1004E000BF0CBE0C031C7E2A4908C5074808031828
:1004F000480FC40747080318470FC307C30CC40CB1
:10050000C50CCD0B6F2AC31B8D2AC50DC40DC30DA1
:10051000C20803199F2AC203400D4C1F9E2A031CC8
:100520009E2AC50F9E2AC40F9E2AC30F9E2A03141B
:10053000C30CC40CC50CC20A0319A22AA92A4C1563
:10054000C201A52ACC14FF30C200C501C40180300D
:10055000C300CE1BAC2AC3134A2AC401C50196307E
:10056000CD00CE13C51FC02AC509C409C309C209DD
:10057000C20FBF2AC30FBF2AC40A0319C50ACE1768
:10058000C5080319DB2A4C1FD22AC51FD22AC30F64
:10059000D22AC40FD22AC50FD22A0314C50CC40C08
:1005A000C30CCD0A0830CD074308C2004408C3007D
:1005B0004508C400F02AC408031DF02A0830CD0203
:1005C0004308031DEC2A0830CD024208031DEB2A24
:1005D0004508CD00FA2AC201C4004208C300C20186
:1005E000C41BF82A0310C20DC30DC40DCD03F02A9D
:1005F000CE1FC4134208C5004D08C2004408CD00F8
:100600004308C4004D08C3004A2A83014030CC008F
:10061000A0014F3083168500033086000D309B000B
:1006200080309F0007309C00FE3083128A01132126
:1006300040308A0113210E308A01132111308A01C2
:10064000132110308A01132110308A011321103038
:100650008A01132115308A0113210E308A011321DA
:1006600000308A011321FE308A01132148308A01AB
:1006700013210A308A0113210E308A01132111300F
:100680008A01132111308A01132111308A011321AB
:1006900011308A0113210E308A01132100308A01A2
:1006A0001321FE308A01132150308A0113210A30B0
:1006B0008A01132111308A01132111308A0113217B
:1006C00011308A01132111308A01132111308A015E
:1006D00013210E308A01132100308A011321FE30CC
:1006E0008A01132158308A01132104308A01132111
:1006F0000E308A01132104308A01132104308A014B
:10070000132104308A01132104308A0113210E3091
:100710008A01132100308A011321FE308A0113213E
:1007200060308A0113210E308A01132111308A01B1
:10073000132110308A0113210E308A011321013058
:100740008A01132115308A0113210E308A011321E9
:1007500000308A011321FE308A01132168308A019A
:1007600013210E308A01132100308A0113210F302A
:100770008A01132110308A01132117308A011321B5
:1007800011308A0113210F308A01132100308A01B0
:100790001321FE308A01132100308A011321003019
:1007A0008A01132100308A01132109308A011321A3
:1007B00009308A01132109308A0113210E308A0180
:1007C000132108308A01132164308A0181218A01B2
:1007D0002820D601D501D801D701DC01DB01DA01DF
:1007E000D901E001DF01DE01DD01E101E301E50105
:1007F000E401E2018A11BE240730AC00D0308A0146
:1008000082218A0128208030A100C0308A01562030
:1008100043308A01132150308A01132153308A0159
:100820001321C5308A01562043308A0113215030EC
:100830008A0113214D308A011321CA308A015620C2
:1008400006308A01132153308A01132176308A0140
:1008500013212F308A01132168308A0113210330BC
:10086000AC00E830AB000530840002308A0104207F
:10087000D5002C08D6008030A100CF308A01562048
:100880002A308A0113218030A1008A015620A50157
:100890005608B0005508AF008A015D20E30A5508EC
:1008A000D70756080318013ED8073B3063028A1168
:1008B000031D5C2C8A11692432308A018121803029
:1008C000A100CF308A01562020308A0113218A01ED
:1008D000032C8030A1008A0156200530A500E630A7
:1008E0008A0165218030A1008A015620A5015608A1
:1008F000B0005508AF008A015D208030A10085302E
:100900008A015620A5015808B0005708AF008A0197
:100910005D205708C2005808C3008A01AD2211307B
:10092000C900C730C8003A30C7007730C6008A0116
:100930004E224508DC004408DB004308DA00420888
:10094000D9008030A1008A308A0156205C08BD00A1
:100950005B08BC005A08BB005908BA0002308A0183
:100960008C20E301D801D701DC01DB01DA01D901D8
:10097000D601D50132308A01812108001030E20011
:10098000023062028A11031CE12C8030A100013088
:10099000A30062088A0134202A308A0113218030A2
:1009A000A1000130A300620A8A01342020308A01AC
:1009B00013212D308A0181210130E2028A110318AE
:1009C000C02C1030E200043062028A11031C042D96
:1009D0008030A1000130A30062088A013420543025
:1009E0008A0113218030A1000130A300620A8A012C
:1009F000342020308A0113212D308A0181210130D9
:100A0000E2028A110318E32C1030E2000630620281
:100A10008A11031C272D8030A1000130A300620839
:100A20008A01342041308A0113218030A100013035
:100A3000A300620A8A01342020308A0113212D305C
:100A40008A0181210130E2028A110318062D10303B
:100A5000E200083062028A11031C4A2D8030A10096
:100A60000130A30062088A01342032308A01132148
:100A70008030A1000130A300620A8A0134202030B6
:100A80008A0113212D308A0181210130E2028A116D
:100A90000318292D1030E2000A3062028A11031C6B
:100AA0006D2D8030A1000130A30062088A0134203E
:100AB00045308A0113218030A1000130A300620A71
:100AC0008A01342020308A0113212D308A018121AE
:100AD0000130E2028A1103184C2D1030E2000C3074
:100AE00062028A11031C902D8030A1000130A30006
:100AF00062088A01342049308A0113218030A10024
:100B00000130A300620A8A01342020308A011321B7
:100B10002D308A0181210130E2028A1103186F2DE4
:100B20001030E2000E3062028A11031CB32D8030B7
:100B3000A1000130A30062088A0134202A308A0112
:100B400013218030A1000130A300620A8A01342001
:100B500020308A0113212D308A0181210130E202E7
:100B60008A110318922D8030A1008E308A01562000
:100B700020308A0113218A0113210330AC00203078
:100B80008A0182218030A100C0308A0156200530C0
:100B9000A500F7308A01652101308A0113214C300C
:100BA0008A01132100308A01132102308A011321A6
:100BB00043308A01132102308A0113210730AC002F
:100BC000D0308A01822108008A01E42D2000200013
:100BD0002000200020002000200020002000200015
:100BE00020002000200020002000200000005200F3
:100BF0004100440059004100530059004F004E008D
:040C000020000000D0
:02400E00223F4F
:00000001FF
